:020000040000FA
:0400000040EF0CF0D1
:08000800056ED8CF06F0E0CF31
:1000100007F00001E9CF0DF0EACF08F0E1CF09F0D9
:10002000E2CF0AF0D9CF0BF0DACF0CF0F3CF14F017
:10003000F4CF15F0FACF16F000C00FF001C010F0A9
:1000400002C011F003C012F004C013F0F2A82CEFAC
:1000500000F0F2B269EF02F00FC000F010C001F042
:1000600011C002F012C003F013C004F00E8E0DC0D8
:10007000E9FF08C0EAFF09C0E1FF0AC0E2FF0BC0C8
:10008000D9FF0CC0DAFF14C0F3FF15C0F4FF16C08F
:10009000FAFF055007C0E0FF06C0D8FF1000F2CFFE
:1000A0000EF0F29EF76AB80FF66E000EF722090006
:1000B000F5500EBEF28E12000A0D353435202D207B
:1000C0004B657970616420416363657373200A0D29
:1000D0000A0D0000F2CF0EF0F29EF76AEE0FF66EF8
:1000E000000EF7220900F5500EBEF28E12002073AA
:1000F000686966745F63686172200000F2CF0EF079
:10010000F29EF76A160FF66E010EF7220900F550FF
:100110000EBEF28E120020636F6D706172655F63B8
:100120006F6465200000F2CF0EF0F29EF76A400F78
:10013000F66E010EF7220900F5500EBEF28E120087
:10014000206E65775F636F6465200000F2CF0EF06C
:10015000F29EF76A660FF66E010EF7220900F5505F
:100160000EBEF28E1200536C656570696E670000FA
:10017000F2CF0EF0F29EF76A8A0FF66E010EF722AA
:100180000900F5500EBEF28E1200526561647900CE
:10019000F2CF0EF0F29EF76AAA0FF66E010EF7226A
:1001A0000900F5500EBEF28E1200636F64655F4168
:1001B0003D202573200A0D00F2CF0EF0F29EF76A63
:1001C000D20FF66E010EF7220900F5500EBEF28E28
:1001D0001200636F64655F423D202573200A0D00A5
:1001E000F2CF0EF0F29EF76AFA0FF66E010EF722CA
:1001F0000900F5500EBEF28E1200636F64655F4316
:100200003D202573200A0D00F2CF0EF0F29EF76A12
:10021000220FF66E020EF7220900F5500EBEF28E86
:100220001200636F64655F443D202573200A0D0052
:10023000F2CF0EF0F29EF76A4A0FF66E020EF72228
:100240000900F5500EBEF28E1200636F64655F699F
:100250006E3D202573200A0D0000F2CF0EF0F29EB5
:10026000F76A740FF66E020EF7220900F5500EBE03
:10027000F28E1200202A2A636F64655F41206D614F
:100280007463682A2A200000F2CF0EF0F29EF76A0B
:10029000A20FF66E020EF7220900F5500EBEF28E86
:1002A0001200202A2A636F64655F42206D617463C7
:1002B000682A2A200000F2CF0EF0F29EF76AD00FD3
:1002C000F66E020EF7220900F5500EBEF28E1200F5
:1002D000202A2A636F64655F43206D617463682A16
:1002E0002A200000F2CF0EF0F29EF76AFE0FF66EA3
:1002F000020EF7220900F5500EBEF28E1200202ADF
:100300002A636F64655F44206D617463682A2A20E4
:100310000000F2CF0EF0F29EF76A2C0FF66E030E7D
:10032000F7220900F5500EBEF28E1200202A2A6331
:100330006F64655F41206368616E67653F2A2A20AC
:100340000000F2CF0EF0F29EF76A5C0FF66E030E1D
:10035000F7220900F5500EBEF28E1200202A2A6301
:100360006F64655F42206368616E67653F2A2A207B
:100370000000F2CF0EF0F29EF76A8C0FF66E030EBD
:10038000F7220900F5500EBEF28E1200202A2A63D1
:100390006F64655F43206368616E67653F2A2A204A
:1003A0000000F2CF0EF0F29EF76ABC0FF66E030E5D
:1003B000F7220900F5500EBEF28E1200202A2A63A1
:1003C0006F64655F44206368616E67653F2A2A2019
:1003D0000000F2CF0EF0F29EF76AEC0FF66E030EFD
:1003E000F7220900F5500EBEF28E120020656570EE
:1003F000726F6D207265736574200000F2CF0EF08D
:10040000F29EF76A160FF66E040EF7220900F550F9
:100410000EBEF28E1200454550524F4D207265734C
:10042000657420200000F2CF0EF0F29EF76A400FB4
:10043000F66E040EF7220900F5500EBEF28E120081
:1004400020746573745F61637469766174652000FC
:10045000F2CF0EF0F29EF76A6A0FF66E040EF722E4
:100460000900F5500EBEF28E1200546573742041DF
:1004700063746976617465200000F2CF0EF0F29E1D
:10048000F76A940FF66E040EF7220900F5500EBEBF
:10049000F28E1200206D617820747269657320728B
:1004A0006561636865642100F2CF0EF0F29EF76A21
:1004B000C20FF66E040EF7220900F5500EBEF28E42
:1004C000120041636365737320426C6F636B6564F4
:1004D000000081A0438243A206D04390476A466A47
:1004E000456A446A01D04380F2922CEF00F0020189
:1004F0003451000818E2366B356B35512C0803E196
:10050000362D01D010D08284F10E006E002EFED761
:1005100000008294F10E006E002EFED70000352BF5
:10052000D8B4362BEAD73451010816E2366B356B56
:1005300035515E0803E1362D01D00ED08284E90EDC
:10054000006E002EFED78294E90E006E002EFED7BC
:10055000352BD8B4362BECD73451020818E2366B61
:10056000356B3551580803E13651020810E082849A
:10057000E00E006E002EFED700D08294E00E006EDA
:10058000002EFED700D0352BD8B4362BEAD7000189
:10059000000CF2CF30F2F29EA96AA69CA69EA6801D
:1005A000A850020130BFF28EFF0851E1A96A340E53
:1005B000A86EA69CA69EA684F2CF00F0F29E0F0124
:1005C000550EA76EAA0EA76EA682A6B2FED7A69457
:1005D0000050F212010EA96E370EA86EA69CA69EC0
:1005E000A684F2CF00F0F29E550EA76EAA0EA76E5B
:1005F000A682A6B2FED7A6940050F212020EA96EF1
:10060000310EA86EA69CA69EA684F2CF00F0F29EA4
:10061000550EA76EAA0EA76EA682A6B2FED7A69406
:100620000050F212030EA96E310EA86EA69CA69E73
:10063000A684F2CF00F0F29E550EA76EAA0EA76E0A
:10064000A682A6B2FED7A6940050F2120201F2CF03
:1006500030F2F29E040EA96EA69CA69EA680A8501B
:1006600030BFF28EFF0852E1040EA96E380EA86E5C
:10067000A69CA69EA684F2CF00F0F29E0F01550E16
:10068000A76EAA0EA76EA682A6B2FED7A6940050A9
:10069000F212050EA96E340EA86EA69CA69EA68424
:1006A000F2CF00F0F29E550EA76EAA0EA76EA6829C
:1006B000A6B2FED7A6940050F212060EA96E310E15
:1006C000A86EA69CA69EA684F2CF00F0F29E550EC0
:1006D000A76EAA0EA76EA682A6B2FED7A694005059
:1006E000F212070EA96E310EA86EA69CA69EA684D5
:1006F000F2CF00F0F29E550EA76EAA0EA76EA6824C
:10070000A6B2FED7A6940050F2120201F2CF30F248
:10071000F29E080EA96EA69CA69EA680A85030BF89
:10072000F28EFF0852E1080EA96E340EA86EA69C48
:10073000A69EA684F2CF00F0F29E0F01550EA76E82
:10074000AA0EA76EA682A6B2FED7A6940050F212F9
:10075000090EA96E370EA86EA69CA69EA684F2CF9F
:1007600000F0F29E550EA76EAA0EA76EA682A6B244
:10077000FED7A6940050F2120A0EA96E320EA86E91
:10078000A69CA69EA684F2CF00F0F29E550EA76E00
:10079000AA0EA76EA682A6B2FED7A6940050F212A9
:1007A0000B0EA96E320EA86EA69CA69EA684F2CF52
:1007B00000F0F29E550EA76EAA0EA76EA682A6B2F4
:1007C000FED7A6940050F2120201F2CF30F2F29E50
:1007D0000C0EA96EA69CA69EA680A85030BFF28ED5
:1007E000FF0852E10C0EA96E380EA86EA69CA69EBC
:1007F000A684F2CF00F0F29E0F01550EA76EAA0E4E
:10080000A76EA682A6B2FED7A6940050F2120D0ED5
:10081000A96E340EA86EA69CA69EA684F2CF00F008
:10082000F29E550EA76EAA0EA76EA682A6B2FED79E
:10083000A6940050F2120E0EA96E320EA86EA69C5F
:10084000A69EA684F2CF00F0F29E550EA76EAA0EC9
:10085000A76EA682A6B2FED7A6940050F2120F0E83
:10086000A96E320EA86EA69CA69EA684F2CF00F0BA
:10087000F29E550EA76EAA0EA76EA682A6B2FED74E
:10088000A6940050F21202012F6B2F51040851E080
:10089000036A2F511E0FE96E000E0320EA6EF2CF9D
:1008A00032F2F29E2FC2A9FFA69CA69EA680A85057
:1008B00032BFF28EEF6E036A2F51230FE96E000EE6
:1008C0000320EA6E040E2F25F2CF33F2F29EA96EBA
:1008D000A69CA69EA680A85033BFF28EEF6E036A38
:1008E0002F51280FE96E000E0320EA6E080E2F2507
:1008F000F2CF33F2F29EA96EA69CA69EA680A850C7
:1009000033BFF28EEF6E036A2F512D0FE96E000E8A
:100910000320EA6E0C0E2F25F2CF33F2F29EA96E61
:10092000A69CA69EA680A85033BFF28EEF6E2F2BFA
:10093000ACD7306B305100012BDC0201302B006E44
:1009400000509EA8FED7AD6E080E305DF3E1EA6A56
:100950001E0EE96E000EEF1008E09EA8FED7EFCF46
:10096000ADFFE92AD8B4EA2AF5D7200E9EA8FED713
:10097000AD6E0A0E9EA8FED7AD6E0D0E9EA8FED7D8
:10098000AD6E306B3051000117DC0201302B006E70
:1009900000509EA8FED7AD6E080E305DF3E1EA6A06
:1009A000230EE96E000EEF1008E09EA8FED7EFCFF1
:1009B000ADFFE92AD8B4EA2AF5D7200E9EA8FED7C3
:1009C000AD6E0A0E9EA8FED7AD6E0D0E9EA8FED788
:1009D000AD6E306B3051000103DC0201302B006E34
:1009E00000509EA8FED7AD6E080E305DF3E1EA6AB6
:1009F000280EE96E000EEF1008E09EA8FED7EFCF9C
:100A0000ADFFE92AD8B4EA2AF5D7200E9EA8FED772
:100A1000AD6E0A0E9EA8FED7AD6E0D0E9EA8FED737
:100A2000AD6E306B3051000104EC01F00201302B4F
:100A3000006E00509EA8FED7AD6E080E305DF2E14C
:100A4000EA6A2D0EE96E000EEF1008E09EA8FED7B0
:100A5000EFCFADFFE92AD8B4EA2AF5D7200E9EA839
:100A6000FED7AD6E0A0E9EA8FED7AD6E0D0E9EA8E7
:100A7000FED7AD6E0001C3EF0FF0080E02013B6F11
:100A80003B530CE081963A51800B02E1819801D0F2
:100A900081888186D8903A373B07F2D70001000C55
:100AA000819A819C36C23AF2E8DF818C000C020107
:100AB0003451070B4009356F366F0001F1DF020139
:100AC00033517F0B8009356F366F0001E9DF000C71
:100AD000818A819C39C23AF2D0DF818C000C495066
:100AE0001F0801E336D049507F0801E232D0486A3E
:100AF000485004082AE349504F0810E34950E00FDA
:100B0000050DF3CF4AF048504A24036A4F0FE96EAF
:100B1000000E0320EA6EEFCF4BF012D049504F0881
:100B20000FE24950B00F050DF3CF4AF048504A2468
:100B3000036A3F0FE96E010E0320EA6EEFCF4BF020
:100B40004BC039F2C5DF482AD3D70201396B000107
:100B5000BFDFAEEF05F038C249F0C1D7000C020E7E
:100B6000EA6E350EE96EEF500DE0060E016E006A7A
:100B7000002EFED7012EFBD77B0E006E002EFED777
:100B8000EF2EF3D7000CEACF37F2E9CF36F20201AD
:100B90003039F009326F3227E20F336F320F356F81
:100BA00030510F0B332733273527E90F346F3427A4
:100BB00034272F390F0B3427352734373537351F76
:100BC00035372F510F0B35273237070E316F0A0E8D
:100BD00034073527FDE333073427FDE33207332796
:100BE000FDE331073227FDE3020EEA6E310EE96EB6
:100BF000070E3615369DE926350EE95CD8B4368DDC
:100C0000EF50006E08E136BD06D036B915D036B7C4
:100C100002D0200E03D036873699300E0026EACF58
:100C200030F2E9CF2FF200C038F2000194DF30C279
:100C3000EAFF2FC2E9FF0201EE5036ADDDD7000119
:100C4000AAEF06F047520DE1465006080BE2FF0AF4
:100C500008E14550A00806E2FF0A03E144502008DD
:100C6000D8A0438043A033D00201336B020E346F0F
:100C700000011DDF02012F6B2F510001A6EC00F0D7
:100C800002012F2B006E386F000165DF080E020194
:100C90002F5DF2E1030E306F2E0E386F00015BDF27
:100CA0000201302FF9D7030E316F200E386F00018B
:100CB00052DF0201312FF9D7C80E356F00014FDF27
:100CC000240E0201366F0001EBDE030049D043B071
:100CD00047D044523FE145523DE146523BE1475245
:100CE00039E1200E0201366F0001DADE0201336BBA
:100CF000020E346F0001DBDE02012F6B2F51000169
:100D0000B8EC00F002012F2B006E386F000123DFDA
:100D1000050E02012F5DF2E1030E306F2E0E386FCB
:100D2000000119DF0201302FF9D7060E316F200EB6
:100D3000386F000110DF0201312FF9D7336B030E3A
:100D4000346F0001B4DE100EE96E42C030F241C0D3
:100D50002FF219D7010E4426000E452246224722C3
:100D6000D6EF0FF084928490020E0201346F0001DE
:100D700077EC02F00201312D13D0848233C234F2B9
:100D8000342B3407D8B406D0FF0E356F0001E7DEF0
:100D90000201F7D732C235F20001E1DE15D00201BF
:100DA0003151020812E1848033C234F2342B34070B
:100DB000D8B406D0FF0E356F0001D1DE0201F7D79F
:100DC00032C235F20001CBDE020184928490010E22
:100DD0004126000E42220001000C80BADBD0020145
:100DE000306B2F6B80BA12D02F2BD8B4302B010E62
:100DF000356F0001B4DE02013051120806E2FF0A2D
:100E000003E12F518708D8A001D0ECD73051120848
:100E1000D8B082D0FF0A04E12F518708D8B07CD027
:100E2000316B31510001E9EC01F00201312B006E10
:100E300000509EA8FED7AD6E0E0E315DF2E1336B11
:100E4000050E346F000133DE0201316B31510001B8
:100E5000FEEC01F00201312B006E386F00017BDEE9
:100E60000E0E0201315DF2E1030E346F000177ECEA
:100E700002F0A96AFF0EA86EA69CA69EA684F2CFD9
:100E800000F0F29E0F01550EA76EAA0EA76EA68265
:100E9000A6B2FED7A6940050F212040EA96EFF0E61
:100EA000A86EA69CA69EA684F2CF00F0F29E550ED8
:100EB000A76EAA0EA76EA682A6B2FED7A694005071
:100EC000F212080EA96EFF0EA86EA69CA69EA6841E
:100ED000F2CF00F0F29E550EA76EAA0EA76EA68264
:100EE000A6B2FED7A6940050F2120C0EA96EFF0E09
:100EF000A86EA69CA69EA684F2CF00F0F29E550E88
:100F0000A76EAA0EA76EA682A6B2FED7A694005020
:100F1000F212FF003ED002013051130839E303E121
:100F20002F51870835E3316B3151000113EC02F08A
:100F30000201312B006E00509EA8FED7AD6E0F0E41
:100F4000315DF2E1336B050E346F0001B0DD02015B
:100F5000316B3151000128EC02F00201312B006E9F
:100F6000386F0001F8DD0E0E0201315DF2E1020E74
:100F7000316F050E336FDC0E326F0001F3DE010EB0
:100F80000201316F050E336FDC0E326F0001EADEB5
:100F90000F01000180BA06D00A0E0201356F000170
:100FA000DEDDF8D7D8EF0FF0210E02012F6F3F0ED4
:100FB000306F326B316B31510A0803E13253D8B4D0
:100FC000C7D08398838A838C050E356F0001C7DDF7
:100FD00081B037D08350070B02012F6F2F510708C4
:100FE00003E1310E306F27D02F51060803E1340E94
:100FF000306F21D02F51050803E1370E306F1BD021
:101000002F51040803E12A0E306F15D02F51030829
:1010100003E1310E306F0FD02F51020803E1340E7F
:10102000306F09D02F2D03D0370E306F04D02F53DF
:1010300002E12A0E306F010E346F000177EC02F0EE
:1010400088D08388839A838C050E0201356F000156
:1010500086DD81B037D08350070B02012F6F2F51EF
:10106000070803E1320E306F27D02F51060803E145
:10107000350E306F21D02F51050803E1380E306F47
:101080001BD02F51040803E1300E306F15D02F51C3
:10109000030803E1320E306F0FD02F51020803E135
:1010A000350E306F09D02F2D03D0380E306F04D09D
:1010B0002F5302E1300E306F010E346F000177ECD8
:1010C00002F047D08388838A839C050E0201356F26
:1010D000000145DD81B037D08350070B02012F6F2F
:1010E0002F51070803E1330E306F27D02F51060828
:1010F00003E1360E306F21D02F51050803E1390E80
:10110000306F1BD02F51040803E1230E306F15D030
:101110002F51030803E1330E306F0FD02F51020817
:1011200003E1360E306F09D02F2D03D0390E306F0A
:1011300004D02F5302E1230E306F010E346F0001F3
:1011400077EC02F006D00201312BD8B4322B33D722
:1011500000013A5005082CE20201336B33510001C3
:101160003DEC02F00201332B006E00509EA8FED72A
:10117000AD6E130E335DF2E1336B050E346F00017B
:1011800096DC0201336B3351000154EC02F0020192
:10119000332B006E386F0001DEDC0E0E0201335D72
:1011A000F2E12D0E306F010E346F000177EC02F08A
:1011B0008398839A839C020130C201F000013EEFC4
:1011C00009F0EACF37F2E9CF36F202013039F009FF
:1011D000326F3227E20F336F320F356F30510F0B02
:1011E000332733273527E90F346F342734272F3936
:1011F0000F0B3427352734373537351F35372F5107
:101200000F0B35273237070E316F0A0E340735279B
:10121000FDE333073427FDE332073327FDE33107CE
:101220003227FDE3020EEA6E310EE96E070E361527
:10123000369DE926350EE95CD8B4368DEF50006E48
:1012400008E136BD06D036B90CD036B702D0200E34
:1012500003D036873699300E002600509EA8FED760
:10126000AD6EEE5036ADE6D7000177EF09F0396A82
:10127000386AFF0E376E81B03ED096D601C037F087
:10128000200E9EA8FED7AD6E37509EA8FED7AD6E3D
:1012900081B022D0140E0201356F000160DC382AC3
:1012A000D8B4392A395203E13850630814E2375070
:1012B0002A0803E03750230806E1030E0201346FC9
:1012C000000177EC02F081B006D0140E0201356FF8
:1012D000000145DCF8D7DCD73A0E9EA8FED7AD6EEC
:1012E000100EE96E39C030F238C02FF26AD7200EE6
:1012F0009EA8FED7AD6EDAEF0FF033C032F034C0E7
:1013000033F035C034F037C035F0F3EF0FF00201A1
:10131000345340E030C2E9FF31C2EAFFEFCF35F28B
:1013200033C203F032C2E9FF33C2EAFFEF50355D4A
:1013300018E031C203F030C2E9FF31C2EAFFEFCF5B
:1013400035F233C203F032C2E9FF33C2EAFFEF5095
:10135000355D03E2FF0E036E01D0010E016E1CD05D
:101360000BD031C203F030C2E9FF31C2EAFFEF52C5
:1013700003E1000E016E10D031C203F03051302B6A
:10138000D8B4312B33C203F03251322BD8B4332BC3
:101390003407BED7000E016E0001000C3A2A02018C
:1013A0002F6B2F51000118EC01F002012F2B006E62
:1013B00000509EA8FED7AD6E090E2F5DF2E1EA6ADD
:1013C000320EE96E000EEF1008E09EA8FED7EFCFB8
:1013D000ADFFE92AD8B4EA2AF5D7200E9EA8FED799
:1013E000AD6E0A0E9EA8FED7AD6E0D0E9EA8FED75E
:1013F000AD6E316B1E0E306F336B320E326F040EDA
:10140000346F000184DF01C03BF00201316B230E19
:10141000306F336B320E326F040E346F000177DFA2
:1014200001C03CF00201316B280E306F336B320E7D
:10143000326F040E346F00016ADF01C03DF002011B
:10144000316B2D0E306F336B320E326F040E346FF2
:1014500000015DDF01C03EF03B521DE137502A081C
:1014600019E102012F6B2F5100012DEC01F0020157
:101470002F2B006E00509EA8FED7AD6E120E2F5D72
:10148000F2E13A6A020E316F050E336FDC0E326FF5
:10149000000168DC1ED03C521CE137502A0819E1DB
:1014A00002012F6B2F51000144EC01F002012F2BA0
:1014B000006E00509EA8FED7AD6E120E2F5DF2E1B9
:1014C0003A6A020E316F050E336FDC0E326F000187
:1014D00049DC3D521DE13750230819E102012F6B11
:1014E0002F5100015BEC01F002012F2B006E005028
:1014F0009EA8FED7AD6E120E2F5DF2E13A6A010E84
:10150000316F050E336FDC0E326F00012BDC1ED005
:101510003E521CE13750230819E102012F6B2F5175
:10152000000172EC01F002012F2B006E00509EA80A
:10153000FED7AD6E120E2F5DF2E13A6A010E316FE9
:10154000050E336FDC0E326F00010CDCFF0E326EC5
:10155000336E346E356E366A14EF10F03F2CC9D0FE
:101560003A2A0201306B3051000118EC01F00201FF
:10157000302B006E00509EA8FED7AD6E090E305D78
:10158000F2E1EA6A320EE96E000EEF1008E09EA862
:10159000FED7EFCFADFFE92AD8B4EA2AF5D7200E5F
:1015A0009EA8FED7AD6E0A0E9EA8FED7AD6E0D0E9C
:1015B0009EA8FED7AD6E316B1E0E306F336B320EB0
:1015C000326F040E346F0001A2DE01C03BF0020155
:1015D000316B230E306F336B320E326F040E346F6B
:1015E000000195DE01C03CF00201316B280E306F26
:1015F000336B320E326F040E346F000188DE01C08F
:101600003DF00201316B2D0E306F336B320E326FB5
:10161000040E346F00017BDE01C03EF03B5219E145
:1016200037502A0815E10201306B3051000189EC76
:1016300001F00201302B006E00509EA8FED7AD6E67
:10164000140E305DF2E1020E3F6E410E406E00015D
:101650001AD03C5218E137502A0815E10201306BCC
:1016600030510001A1EC01F00201302B006E00505E
:101670009EA8FED7AD6E140E305DF2E1020E3F6EF5
:10168000420E406E00013D5219E13750230815E12A
:101690000201306B30510001B9EC01F00201302B36
:1016A000006E00509EA8FED7AD6E140E305DF2E1C4
:1016B000020E3F6E430E406E00011AD03E5218E1FA
:1016C0003750230815E10201306B30510001D1EC95
:1016D00001F00201302B006E00509EA8FED7AD6EC7
:1016E000140E305DF2E1020E3F6E440E406E0001BA
:1016F000C6D03F500208D8A4C2D04050410828E1CB
:1017000002012F6B2F51040821E0036A2F51320F81
:10171000E96E000E0320EA6EEFCF30F22FC2A9FF70
:1017200030C2A8FFA69CA69EA684F2CF00F0F29E2F
:101730000F01550EA76EAA0EA76EA682A6B2FED7FF
:10174000A6940050F21202012F2BDCD789D00001A1
:10175000405042082BE102012F6B2F51040824E076
:10176000040E2F25306F036A2F51320FE96E000EE1
:101770000320EA6EEFCF31F230C2A9FF31C2A8FFD9
:10178000A69CA69EA684F2CF00F0F29E0F01550EF5
:10179000A76EAA0EA76EA682A6B2FED7A694005088
:1017A000F21202012F2BD9D75BD000014050430821
:1017B0002BE102012F6B2F51040824E0080E2F2586
:1017C000306F036A2F51320FE96E000E0320EA6E6C
:1017D000EFCF31F230C2A9FF31C2A8FFA69CA69E6E
:1017E000A684F2CF00F0F29E0F01550EA76EAA0E4E
:1017F000A76EA682A6B2FED7A6940050F2120201EE
:101800002F2BD9D72DD000014050440829E10201E7
:101810002F6B2F51040824E00C0E2F25306F036A24
:101820002F51320FE96E000E0320EA6EEFCF31F236
:1018300030C2A9FF31C2A8FFA69CA69EA684F2CF03
:1018400000F0F29E0F01550EA76EAA0EA76EA6829B
:10185000A6B2FED7A6940050F21202012F2BD9D7C0
:10186000030E0201346F000177EC02F0030E020157
:10187000346F000177EC02F0FF00010E3F6E000CA8
:10188000F86AD09E0D8EFE0E006E060E016E020EE0
:10189000E96E000EEA6EEE6A002EFDD7012EFBD730
:1018A000EA6AE96A0A0EAF6EA60EAC6E900EAB6ED7
:1018B000C180C182C184C196186A196A4F6A506A90
:1018C000516A526A536A546A556A5F0E566E576A75
:1018D000586A596A070E5A6E5B6A5C6E5D6A140E2E
:1018E0005E6E7F0E5F6E140E606E7F0E616E140E64
:1018F000626E240E636E2A0E646E7F0E656E2A0E73
:10190000666E120E676E230E686E130E696E080EF9
:101910006A6E640E6B6E620E6C6E360E6D6E490EE4
:101920006E6E550E6F6E220E706E500E716E726A74
:10193000050E736E030E746E756A766A776A1C0EF6
:10194000786E220E796E410E7A6E7B6A7C6A7D6EAD
:10195000220E7E6E1C0E7F6E806B140E816F080E41
:10196000826F3E0E836F080E846F140E856F080E13
:10197000866F876F3E0E886F080E896F8A6F8B6B3C
:10198000500E8C6F300E8D6F8E6B8F6B080E906FBC
:10199000916F926F936F946F956B600E966F976FC8
:1019A000986B996B200E9A6F100E9B6F080E9C6FB0
:1019B000040E9D6F020E9E6F3E0E9F6F510EA06F24
:1019C000490EA16F450EA26F3E0EA36FA46B420E8F
:1019D000A56F7F0EA66F400EA76FA86B420EA96F72
:1019E000610EAA6F510EAB6F490EAC6F460EAD6F14
:1019F000210EAE6F410EAF6F450EB06F4B0EB16F43
:101A0000310EB26F180EB36F140EB46F120EB56FA5
:101A10007F0EB66F100EB76F270EB86F450EB96FF9
:101A2000BA6FBB6F390EBC6F3C0EBD6F4A0EBE6FF6
:101A3000490EBF6FC06F300EC16F010EC26F710EC5
:101A4000C36F090EC46F050EC56F030EC66F360E49
:101A5000C76F490EC86FC96FCA6F360ECB6F060EBF
:101A6000CC6F490ECD6FCE6F290ECF6F1E0ED06F8B
:101A7000D16B360ED26FD36FD46BD56BD66B560E3F
:101A8000D76F360ED86FD96BDA6B080EDB6F140E7A
:101A9000DC6F220EDD6F410EDE6FDF6B140EE06F28
:101AA000E16FE26FE36FE46FE56B410EE66F220ECC
:101AB000E76F140EE86F080EE96F020EEA6F010E71
:101AC000EB6F510EEC6F090EED6F060EEE6F320EDE
:101AD000EF6F490EF06F790EF16F410EF26F3E0E0F
:101AE000F36F7E0EF46F110EF56FF66FF76F7E0ECB
:101AF000F86F7F0EF96F490EFA6FFB6FFC6F360EB1
:101B0000FD6F3E0EFE6F410EFF6F0101006F016F12
:101B1000220E026F7F0E036F410E046F056F220EBF
:101B2000066F1C0E076F7F0E086F490E096F0A6F54
:101B30000B6F410E0C6F7F0E0D6F090E0E6F0F6F46
:101B4000106F010E116F3E0E126F410E136F490E92
:101B5000146F156F7A0E166F7F0E176F080E186FC1
:101B6000196F1A6F7F0E1B6F1C6B410E1D6F7F0E5E
:101B70001E6F410E1F6F206B200E216F400E226FD3
:101B8000410E236F3F0E246F010E256F7F0E266FCF
:101B9000080E276F140E286F220E296F410E2A6F30
:101BA0007F0E2B6F400E2C6F2D6F2E6F2F6F7F0EC1
:101BB000306F020E316F0C0E326F020E336F7F0EDC
:101BC000346F356F040E366F080E376F100E386F96
:101BD0007F0E396F3E0E3A6F410E3B6F3C6F3D6F8B
:101BE0003E0E3E6F7F0E3F6F090E406F416F426F9A
:101BF000060E436F3E0E446F410E456F510E466F09
:101C0000210E476F5E0E486F7F0E496F090E4A6FB7
:101C1000190E4B6F290E4C6F460E4D6F4E6F490ECD
:101C20004F6F506F516F310E526F010E536F546FE3
:101C30007F0E556F010E566F576F3F0E586F400E57
:101C4000596F5A6F5B6F3F0E5C6F1F0E5D6F200EFA
:101C50005E6F400E5F6F200E606F1F0E616F3F0E54
:101C6000626F400E636F380E646F400E656F3F0EFB
:101C7000666F630E676F140E686F080E696F140E3F
:101C80006A6F630E6B6F070E6C6F080E6D6F700ED0
:101C90006E6F080E6F6F070E706F610E716F510ED1
:101CA000726F490E736F450E746F430E756F766BCE
:101CB0007F0E776F410E786F796F7A6B020E7B6FB4
:101CC000040E7C6F080E7D6F100E7E6F200E7F6FEE
:101CD000806B410E816F826F7F0E836F846B040E69
:101CE000856F020E866F010E876F020E886F040EDD
:101CF000896F400E8A6F8B6F8C6F8D6F8E6F8F6BBD
:101D0000010E906F020E916F040E926F936B200E76
:101D1000946F540E956F966F976F780E986F7F0E35
:101D2000996F480E9A6F440E9B6F9C6F380E9D6F93
:101D30009E6F440E9F6FA06FA16F200EA26F380E92
:101D4000A36F440EA46FA56F480EA66F7F0EA76FFA
:101D5000380EA86F540EA96FAA6FAB6F180EAC6F38
:101D6000080EAD6F7E0EAE6F090EAF6F010EB06F35
:101D7000020EB16F0C0EB26F520EB36FB46FB56F2F
:101D80003E0EB66F7F0EB76F080EB86F040EB96FB8
:101D9000BA6F780EBB6FBC6B440EBD6F7D0EBE6F0D
:101DA000400EBF6FC06B200EC16F400EC26F440E5D
:101DB000C36F3D0EC46FC56B7F0EC66F100EC76F2D
:101DC000280EC86F440EC96FCA6BCB6B410ECC6F27
:101DD0007F0ECD6F400ECE6FCF6B7C0ED06F040E9A
:101DE000D16F180ED26F040ED36F780ED46F7C0EA5
:101DF000D56F080ED66F040ED76FD86F780ED96FD7
:101E0000380EDA6F440EDB6FDC6FDD6F380EDE6F7D
:101E10007C0EDF6F140EE06FE16FE26F080EE36F70
:101E2000E46F140EE56FE66F180EE76F7C0EE86F37
:101E3000E96F080EEA6F040EEB6FEC6F080EED6FA2
:101E4000480EEE6F540EEF6FF06FF16F200EF26FD1
:101E5000040EF36F3F0EF46F440EF56F400EF66FF5
:101E6000200EF76F3C0EF86F400EF96FFA6F200EE0
:101E7000FB6F7C0EFC6F1C0EFD6F200EFE6F400E84
:101E8000FF6F200E0201006F1C0E016F3C0E026FEF
:101E9000400E036F300E046F400E056F3C0E066F50
:101EA000440E076F280E086F100E096F280E0A6F78
:101EB000440E0B6F0C0E0C6F500E0D6F0E6F0F6FEC
:101EC0003C0E106F440E116F640E126F540E136FA0
:101ED0004C0E146F440E156F166B080E176F360EEE
:101EE000186F410E196F1A6B1B6B1C6B7F0E1D6FE9
:101EF0001E6B1F6B206B410E216F360E226F080E7A
:101F0000236F246B100E256F080E266F276F100E9F
:101F1000286F080E296F780E2A6F460E2B6F410E20
:101F20002C6F460E2D6F780E2E6F43924390F19CCE
:101F3000F288C00EF212C290C180C182C184C196E3
:101F4000200E926E010E936E800E946E070E956EAB
:101F5000969096929684010E346F000177EC02F011
:101F600002012F6B2F5100014FEC00F002012F2BCB
:101F7000006E00509EA8FED7AD6E1A0E2F5DF2E1E6
:101F80000001C9EF02F0020E0201346F000177EC8C
:101F900002F03A6AFF0E326E336E346E356E366A78
:101FA000010E3F6E426A416A22EF06F0EDEF06F045
:101FB00037EF09F037502F0817E23750390814E38C
:101FC00002012F6B2F5100016AEC00F002012F2B50
:101FD000006E00509EA8FED7AD6E0C0E2F5DF2E194
:101FE00000017DEF09F03FD037502A0803E0375059
:101FF000230839E13F2C32D0395217E138506308B9
:1020000014E302012F6B2F5100017EEC00F002015E
:102010002F2B006E00509EA8FED7AD6E0E0E2F5DCA
:10202000F2E10001CEEF09F018D0395203E1385047
:10203000630813E202012F6B2F51000193EC00F0B3
:1020400002012F2B006E00509EA8FED7AD6E0A0E27
:102050002F5DF2E10001AEEC0AF005D03F5002081E
:0A20600002E1AEEC0AF0A0D7030085
:020000040030CA
:0E00000000220C0E000180000FC00FE00F4028
:00000001FF
